 gles1_texture_stream

 Timestamp is 4be8c409 (Tue May 11 11:42:17 2010)

 Preferred load address is 00010000

 Start         Length     Name                   Class
 0001:00000000 00000004H .CRT$XCA                CODE
 0001:00000004 00000004H .CRT$XCZ                CODE
 0001:00000008 00000004H .CRT$XIA                CODE
 0001:0000000c 00000004H .CRT$XIZ                CODE
 0001:00000010 00000004H .CRT$XPA                CODE
 0001:00000014 00000004H .CRT$XPZ                CODE
 0001:00000018 00000004H .CRT$XTA                CODE
 0001:0000001c 00000004H .CRT$XTZ                CODE
 0001:00000020 00000580H .rdata                  CODE
 0001:000005a0 00000031H .rdata$debug            CODE
 0001:000005d4 00001240H .text                   CODE
 0001:00001814 00000014H .xdata                  CODE
 0001:00001828 00000028H .idata$2                CODE
 0001:00001850 00000014H .idata$3                CODE
 0001:00001864 000000f8H .idata$4                CODE
 0001:0000195c 0000001cH .idata$6                CODE
 0001:00001978 00000000H .edata                  CODE
 0002:00000000 000000f8H .idata$5                DATA
 0002:000000f8 0002ab18H .data                   DATA
 0002:0002ac10 0000004cH .bss                    DATA
 0003:00000000 00000090H .pdata                  DATA

  Address         Publics by Value              Rva+Base       Lib:Object

 0000:00000000       ___safe_se_handler_table   00000000     <absolute>
 0000:00000000       ___safe_se_handler_count   00000000     <absolute>
 0001:00000000       __xc_a                     00011000     corelib0:crt0init.obj
 0001:00000004       __xc_z                     00011004     corelib0:crt0init.obj
 0001:00000008       __xi_a                     00011008     corelib0:crt0init.obj
 0001:0000000c       __xi_z                     0001100c     corelib0:crt0init.obj
 0001:00000010       __xp_a                     00011010     corelib0:crt0init.obj
 0001:00000014       __xp_z                     00011014     corelib0:crt0init.obj
 0001:00000018       __xt_a                     00011018     corelib0:crt0init.obj
 0001:0000001c       __xt_z                     0001101c     corelib0:crt0init.obj
 0001:0000003c       ??_C@_0CP@IHJEEKMK@?$CB?$CB?$CB?$CB?5?5CreateFile?5failed?5?3?5GetLas@ 0001103c     example_bufferclass_ctrl_wince.obj
 0001:0000006c       ??_C@_1M@BMDCKMBI@?$AAB?$AAC?$AAE?$AA1?$AA?3?$AA?$AA@ 0001106c     example_bufferclass_ctrl_wince.obj
 0001:00000078       ??_C@_17NEGDDFML@?$AAB?$AAC?$AAE?$AA?$AA@ 00011078     example_bufferclass_ctrl_wince.obj
 0001:00000080       ??_C@_1O@GBAEOCCH@?$AAP?$AAr?$AAe?$AAf?$AAi?$AAx?$AA?$AA@ 00011080     example_bufferclass_ctrl_wince.obj
 0001:00000090       ??_C@_1BO@DKFMECLO@?$AAb?$AAc?$AA_?$AAe?$AAx?$AAa?$AAm?$AAp?$AAl?$AAe?$AA?4?$AAd?$AAl?$AAl?$AA?$AA@ 00011090     example_bufferclass_ctrl_wince.obj
 0001:000000b0       ??_C@_17DJMMGLBL@?$AAD?$AAl?$AAl?$AA?$AA@ 000110b0     example_bufferclass_ctrl_wince.obj
 0001:000000b8       ??_C@_19NBCCPLHE@?$AAK?$AAe?$AAe?$AAp?$AA?$AA@ 000110b8     example_bufferclass_ctrl_wince.obj
 0001:000000c4       ??_C@_1CG@CKALJGDC@?$AA?2?$AAP?$AAo?$AAw?$AAe?$AAr?$AAV?$AAR?$AA?2?$AAB?$AAC?$AAE?$AAx?$AAa?$AAm?$AAp?$AAl?$AAe?$AA?$AA@ 000110c4     example_bufferclass_ctrl_wince.obj
 0001:000000ec       ??_C@_0DG@HMPOADHB@?9?9?9?9?9?9?9?9?9?9?9?9?9?9?9?9?9?9?9?9?9?5finished?5?9@ 000110ec     example_bufferclass_ctrl_wince.obj
 0001:00000128       ??_C@_0FC@NALJDPJ@Capture?5buffers?5Count?5?$CFd?5doesn?8t@ 00011128     example_bufferclass_ctrl_wince.obj
 0001:0000017c       ??_C@_0CL@IANBJKLB@no?5capture?5buffers?5available?5?9?5e@ 0001117c     example_bufferclass_ctrl_wince.obj
 0001:000001a8       ??_C@_0BP@BPDGIKFD@?$CB?$CB?$CB?$CB?5?5DeviceIoControl?5failed?5?6?$AA@ 000111a8     example_bufferclass_ctrl_wince.obj
 0001:000001c8       ??_C@_0DF@DFKFEDON@?9?9?9?9?9?9?9?9?9?9?9?9?9?9?9?9?9?9?9?9?9?5started?5?9?9@ 000111c8     example_bufferclass_ctrl_wince.obj
 0001:00000200       ??_C@_0BA@ECMACICF@EGL_BAD_SURFACE?$AA@ 00011200     example_bufferclass_draw.obj
 0001:00000210       ??_C@_0BC@OMABNJPB@EGL_BAD_PARAMETER?$AA@ 00011210     example_bufferclass_draw.obj
 0001:00000224       ??_C@_0BG@JCAPPMPM@EGL_BAD_NATIVE_WINDOW?$AA@ 00011224     example_bufferclass_draw.obj
 0001:0000023c       ??_C@_0BG@IANPFEBH@EGL_BAD_NATIVE_PIXMAP?$AA@ 0001123c     example_bufferclass_draw.obj
 0001:00000254       ??_C@_0O@GCFMIHO@EGL_BAD_MATCH?$AA@ 00011254     example_bufferclass_draw.obj
 0001:00000264       ??_C@_0BA@KHKFAGME@EGL_BAD_DISPLAY?$AA@ 00011264     example_bufferclass_draw.obj
 0001:00000274       ??_C@_0BI@KBFIGPCO@EGL_BAD_CURRENT_SURFACE?$AA@ 00011274     example_bufferclass_draw.obj
 0001:0000028c       ??_C@_0BA@FPCJCEFK@EGL_BAD_CONTEXT?$AA@ 0001128c     example_bufferclass_draw.obj
 0001:0000029c       ??_C@_0P@HOPKKPDK@EGL_BAD_CONFIG?$AA@ 0001129c     example_bufferclass_draw.obj
 0001:000002ac       ??_C@_0BC@NLAJAPHP@EGL_BAD_ATTRIBUTE?$AA@ 000112ac     example_bufferclass_draw.obj
 0001:000002c0       ??_C@_0O@PGDEJDGL@EGL_BAD_ALLOC?$AA@ 000112c0     example_bufferclass_draw.obj
 0001:000002d0       ??_C@_0P@ELJNOEME@EGL_BAD_ACCESS?$AA@ 000112d0     example_bufferclass_draw.obj
 0001:000002e0       ??_C@_0BE@JIJLFFAN@EGL_NOT_INITIALIZED?$AA@ 000112e0     example_bufferclass_draw.obj
 0001:000002f4       ??_C@_0M@JFIJMCIK@EGL_SUCCESS?$AA@ 000112f4     example_bufferclass_draw.obj
 0001:00000338       ??_C@_0EK@HNEICOHN@?6Stream?5Device?5?$CFs?3?5numBuffers?5?$DN?5@ 00011338     example_bufferclass_draw.obj
 0001:00000384       ??_C@_0BD@PIBFHNP@glTexBindStreamIMG?$AA@ 00011384     example_bufferclass_draw.obj
 0001:00000398       ??_C@_0CD@OCNNIBKN@glGetTexStreamDeviceAttributeivI@ 00011398     example_bufferclass_draw.obj
 0001:000003bc       ??_C@_0BM@MBNDOCOP@glGetTexStreamDeviceNameIMG?$AA@ 000113bc     example_bufferclass_draw.obj
 0001:000003d8       ??_C@_0BG@IMEBFAFH@GL_IMG_texture_stream?$AA@ 000113d8     example_bufferclass_draw.obj
 0001:000003f0       ??_C@_0CF@GLNKALBC@?8?$CFs?8?5returned?5egl?5error?5?8?$CFs?8?5?$CI0x@ 000113f0     example_bufferclass_draw.obj
 0001:00000418       ??_C@_0P@PNPBPNLI@eglMakeCurrent?$AA@ 00011418     example_bufferclass_draw.obj
 0001:00000428       ??_C@_0BB@KEKMNHDF@eglCreateContext?$AA@ 00011428     example_bufferclass_draw.obj
 0001:0000043c       ??_C@_0BH@MDMCFBDG@eglCreateWindowSurface?$AA@ 0001143c     example_bufferclass_draw.obj
 0001:00000454       ??_C@_0BA@GKADIFMO@eglChooseConfig?$AA@ 00011454     example_bufferclass_draw.obj
 0001:00000464       ??_C@_0O@OMNEJBKO@eglGetConfigs?$AA@ 00011464     example_bufferclass_draw.obj
 0001:00000474       ??_C@_0O@EEJFKEKH@eglInitialize?$AA@ 00011474     example_bufferclass_draw.obj
 0001:00000488       ??_C@_1KE@BDGMONOJ@?$AAH?$AA?3?$AA?2?$AAW?$AAI?$AAN?$AAC?$AAE?$AA6?$AA0?$AA0?$AA?2?$AAP?$AAL?$AAA?$AAT?$AAF?$AAO?$AAR?$AAM?$AA?2?$AAS?$AAM?$AAD?$AAK?$AAV?$AA2?$AA1?$AA0?$AA?2?$AAS?$AAR@ 00011488     wince_unittests.obj
 0001:0000052c       ??_C@_1CI@OHCJFJPM@?$AAE?$AAR?$AAR?$AAO?$AAR?$AA?3?$AA?5?$AA?$CF?$AAs?$AA?5?$AAl?$AAi?$AAn?$AAe?$AA?5?$AA?$CF?$AAd?$AA?3?$AA?5?$AA?$AA@ 0001152c     wince_unittests.obj
 0001:00000554       ??_C@_1CK@MPGKAOE@?$AA?$CI?$AAe?$AAr?$AAr?$AAo?$AAr?$AA?5?$AAc?$AAo?$AAd?$AAe?$AA?3?$AA?5?$AA?$CF?$AAd?$AA?$CJ?$AA?3?$AA?5?$AA?$CF?$AAs?$AA?$AA@ 00011554     wince_unittests.obj
 0001:00000580       ??_C@_1M@DMCDIEDK@?$AAP?$AAK?$AAM?$AA1?$AA?3?$AA?$AA@ 00011580     wince_unittests.obj
 0001:0000058c       ??_C@_0L@GPAGIAIC@?9disablepm?$AA@ 0001158c     wince_unittests.obj
 0001:00000598       ??_C@_07FBLHGNAH@app?4exe?$AA@ 00011598     wince_unittests.obj
 0001:000005d4       _UnloadDriver              000115d4 f   example_bufferclass_ctrl_wince.obj
 0001:00000600       _LoadDriver                00011600 f   example_bufferclass_ctrl_wince.obj
 0001:00000778       main                       00011778 f   example_bufferclass_ctrl_wince.obj
 0001:00000c14       DrawTexStream              00011c14 f   example_bufferclass_draw.obj
 0001:00000d50       DeInitTexStreamDisplay     00011d50 f   example_bufferclass_draw.obj
 0001:00000de4       InitTexStreamDisplay       00011de4 f   example_bufferclass_draw.obj
 0001:00001074       WinMain                    00012074 f   wince_unittests.obj
 0001:0000129c       glGetString                0001229c f   libGLES_CM:libGLES_CM.dll
 0001:000012ac       glTexParameterf            000122ac f   libGLES_CM:libGLES_CM.dll
 0001:000012bc       glTexEnvf                  000122bc f   libGLES_CM:libGLES_CM.dll
 0001:000012cc       glTexImage2D               000122cc f   libGLES_CM:libGLES_CM.dll
 0001:000012dc       glColor4f                  000122dc f   libGLES_CM:libGLES_CM.dll
 0001:000012ec       glTexCoordPointer          000122ec f   libGLES_CM:libGLES_CM.dll
 0001:000012fc       glVertexPointer            000122fc f   libGLES_CM:libGLES_CM.dll
 0001:0000130c       glEnableClientState        0001230c f   libGLES_CM:libGLES_CM.dll
 0001:0000131c       glShadeModel               0001231c f   libGLES_CM:libGLES_CM.dll
 0001:0000132c       glClearColor               0001232c f   libGLES_CM:libGLES_CM.dll
 0001:0000133c       glDisable                  0001233c f   libGLES_CM:libGLES_CM.dll
 0001:0000134c       glTranslatef               0001234c f   libGLES_CM:libGLES_CM.dll
 0001:0000135c       glDrawArrays               0001235c f   libGLES_CM:libGLES_CM.dll
 0001:0000136c       glEnable                   0001236c f   libGLES_CM:libGLES_CM.dll
 0001:0000137c       glScalef                   0001237c f   libGLES_CM:libGLES_CM.dll
 0001:0000138c       glLoadIdentity             0001238c f   libGLES_CM:libGLES_CM.dll
 0001:0000139c       glMatrixMode               0001239c f   libGLES_CM:libGLES_CM.dll
 0001:000013ac       glClear                    000123ac f   libGLES_CM:libGLES_CM.dll
 0001:000013bc       DeactivateDevice           000123bc f   coredll:COREDLL.dll
 0001:000013cc       CloseHandle                000123cc f   coredll:COREDLL.dll
 0001:000013dc       GetLastError               000123dc f   coredll:COREDLL.dll
 0001:000013ec       CreateFileW                000123ec f   coredll:COREDLL.dll
 0001:000013fc       Sleep                      000123fc f   coredll:COREDLL.dll
 0001:0000140c       ActivateDevice             0001240c f   coredll:COREDLL.dll
 0001:0000141c       RegCloseKey                0001241c f   coredll:COREDLL.dll
 0001:0000142c       RegSetValueExW             0001242c f   coredll:COREDLL.dll
 0001:0000143c       RegCreateKeyExW            0001243c f   coredll:COREDLL.dll
 0001:0000144c       DeviceIoControl            0001244c f   coredll:COREDLL.dll
 0001:0000145c       ReleasePowerRequirement    0001245c f   coredll:COREDLL.dll
 0001:0000146c       NKDbgPrintfW               0001246c f   coredll:COREDLL.dll
 0001:0000147c       FormatMessageW             0001247c f   coredll:COREDLL.dll
 0001:0000148c       SetPowerRequirement        0001248c f   coredll:COREDLL.dll
 0001:0000149c       WideCharToMultiByte        0001249c f   coredll:COREDLL.dll
 0001:0000152c       WinMainCRTStartup          0001252c f   corelib0:pegwmain.obj
 0001:00001628       exit                       00012628 f   corelib0:cexit.obj
 0001:00001640       _exit                      00012640 f   corelib0:cexit.obj
 0001:00001680       _initterm                  00012680 f   corelib0:crt0dat.obj
 0001:000016b4       _cinit                     000126b4 f   corelib0:crt0dat.obj
 0001:000016e8       __security_init_cookie     000126e8 f   corelib0:seccinit.obj
 0001:00001744       fprintf                    00012744 f   corelib1:COREDLL.dll
 0001:00001754       _getstdfilex               00012754 f   corelib1:COREDLL.dll
 0001:00001764       strstr                     00012764 f   corelib1:COREDLL.dll
 0001:00001774       _stricmp                   00012774 f   corelib1:COREDLL.dll
 0001:00001784       _isctype                   00012784 f   corelib1:COREDLL.dll
 0001:00001794       malloc                     00012794 f   corelib1:COREDLL.dll
 0001:000017a4       wcslen                     000127a4 f   corelib1:COREDLL.dll
 0001:000017b4       memset                     000127b4 f   corelib1:COREDLL.dll
 0001:000017c4       _XcptFilter                000127c4 f   corelib1:COREDLL.dll
 0001:000017d4       __C_specific_handler       000127d4 f   corelib1:COREDLL.dll
 0001:000017e4       free                       000127e4 f   corelib1:COREDLL.dll
 0001:000017f4       __security_gen_cookie2     000127f4 f   corelib1:COREDLL.dll
 0001:00001804       TerminateProcess           00012804 f   coredll:COREDLL.dll
 0001:00001828       __IMPORT_DESCRIPTOR_libGLES_CM 00012828     libGLES_CM:libGLES_CM.dll
 0001:0000183c       __IMPORT_DESCRIPTOR_COREDLL 0001283c     coredll:COREDLL.dll
 0001:00001850       __NULL_IMPORT_DESCRIPTOR   00012850     libGLES_CM:libGLES_CM.dll
 0002:00000000       __imp_DeactivateDevice     00013000     coredll:COREDLL.dll
 0002:00000004       __imp___security_gen_cookie2 00013004     corelib1:COREDLL.dll
 0002:00000008       __imp_free                 00013008     corelib1:COREDLL.dll
 0002:0000000c       __imp___C_specific_handler 0001300c     corelib1:COREDLL.dll
 0002:00000010       __imp__XcptFilter          00013010     corelib1:COREDLL.dll
 0002:00000014       __imp_memset               00013014     corelib1:COREDLL.dll
 0002:00000018       __imp_wcslen               00013018     corelib1:COREDLL.dll
 0002:0000001c       __imp_malloc               0001301c     corelib1:COREDLL.dll
 0002:00000020       __imp__isctype             00013020     corelib1:COREDLL.dll
 0002:00000024       __imp__stricmp             00013024     corelib1:COREDLL.dll
 0002:00000028       __imp_strstr               00013028     corelib1:COREDLL.dll
 0002:0000002c       __imp___rt_udiv            0001302c     corelib1:COREDLL.dll
 0002:00000030       __imp__getstdfilex         00013030     corelib1:COREDLL.dll
 0002:00000034       __imp_fprintf              00013034     corelib1:COREDLL.dll
 0002:00000038       __imp_WideCharToMultiByte  00013038     coredll:COREDLL.dll
 0002:0000003c       __imp_SetPowerRequirement  0001303c     coredll:COREDLL.dll
 0002:00000040       __imp_FormatMessageW       00013040     coredll:COREDLL.dll
 0002:00000044       __imp_NKDbgPrintfW         00013044     coredll:COREDLL.dll
 0002:00000048       __imp_ReleasePowerRequirement 00013048     coredll:COREDLL.dll
 0002:0000004c       __imp_DeviceIoControl      0001304c     coredll:COREDLL.dll
 0002:00000050       __imp_RegCreateKeyExW      00013050     coredll:COREDLL.dll
 0002:00000054       __imp_RegSetValueExW       00013054     coredll:COREDLL.dll
 0002:00000058       __imp_RegCloseKey          00013058     coredll:COREDLL.dll
 0002:0000005c       __imp_ActivateDevice       0001305c     coredll:COREDLL.dll
 0002:00000060       __imp_Sleep                00013060     coredll:COREDLL.dll
 0002:00000064       __imp_CreateFileW          00013064     coredll:COREDLL.dll
 0002:00000068       __imp_GetLastError         00013068     coredll:COREDLL.dll
 0002:0000006c       __imp_CloseHandle          0001306c     coredll:COREDLL.dll
 0002:00000070       __imp_TerminateProcess     00013070     coredll:COREDLL.dll
 0002:00000074       \177COREDLL_NULL_THUNK_DATA 00013074     coredll:COREDLL.dll
 0002:00000078       __imp_eglInitialize        00013078     libGLES_CM:libGLES_CM.dll
 0002:0000007c       __imp_eglGetDisplay        0001307c     libGLES_CM:libGLES_CM.dll
 0002:00000080       __imp_eglGetConfigs        00013080     libGLES_CM:libGLES_CM.dll
 0002:00000084       __imp_eglChooseConfig      00013084     libGLES_CM:libGLES_CM.dll
 0002:00000088       __imp_eglCreateWindowSurface 00013088     libGLES_CM:libGLES_CM.dll
 0002:0000008c       __imp_eglCreateContext     0001308c     libGLES_CM:libGLES_CM.dll
 0002:00000090       __imp_eglTerminate         00013090     libGLES_CM:libGLES_CM.dll
 0002:00000094       __imp_eglDestroySurface    00013094     libGLES_CM:libGLES_CM.dll
 0002:00000098       __imp_eglDestroyContext    00013098     libGLES_CM:libGLES_CM.dll
 0002:0000009c       __imp_eglMakeCurrent       0001309c     libGLES_CM:libGLES_CM.dll
 0002:000000a0       __imp_eglGetError          000130a0     libGLES_CM:libGLES_CM.dll
 0002:000000a4       __imp_eglSwapBuffers       000130a4     libGLES_CM:libGLES_CM.dll
 0002:000000a8       __imp_glClear              000130a8     libGLES_CM:libGLES_CM.dll
 0002:000000ac       __imp_glMatrixMode         000130ac     libGLES_CM:libGLES_CM.dll
 0002:000000b0       __imp_glLoadIdentity       000130b0     libGLES_CM:libGLES_CM.dll
 0002:000000b4       __imp_glScalef             000130b4     libGLES_CM:libGLES_CM.dll
 0002:000000b8       __imp_glEnable             000130b8     libGLES_CM:libGLES_CM.dll
 0002:000000bc       __imp_glDrawArrays         000130bc     libGLES_CM:libGLES_CM.dll
 0002:000000c0       __imp_glTranslatef         000130c0     libGLES_CM:libGLES_CM.dll
 0002:000000c4       __imp_glDisable            000130c4     libGLES_CM:libGLES_CM.dll
 0002:000000c8       __imp_eglGetProcAddress    000130c8     libGLES_CM:libGLES_CM.dll
 0002:000000cc       __imp_glClearColor         000130cc     libGLES_CM:libGLES_CM.dll
 0002:000000d0       __imp_glShadeModel         000130d0     libGLES_CM:libGLES_CM.dll
 0002:000000d4       __imp_glEnableClientState  000130d4     libGLES_CM:libGLES_CM.dll
 0002:000000d8       __imp_glVertexPointer      000130d8     libGLES_CM:libGLES_CM.dll
 0002:000000dc       __imp_glTexCoordPointer    000130dc     libGLES_CM:libGLES_CM.dll
 0002:000000e0       __imp_glColor4f            000130e0     libGLES_CM:libGLES_CM.dll
 0002:000000e4       __imp_glTexImage2D         000130e4     libGLES_CM:libGLES_CM.dll
 0002:000000e8       __imp_glTexEnvf            000130e8     libGLES_CM:libGLES_CM.dll
 0002:000000ec       __imp_glTexParameterf      000130ec     libGLES_CM:libGLES_CM.dll
 0002:000000f0       __imp_glGetString          000130f0     libGLES_CM:libGLES_CM.dll
 0002:000000f4       \177libGLES_CM_NULL_THUNK_DATA 000130f4     libGLES_CM:libGLES_CM.dll
 0002:000000f8       bRender                    000130f8     example_bufferclass_ctrl_wince.obj
 0002:000000fc       hDevice                    000130fc     example_bufferclass_ctrl_wince.obj
 0002:00000100       hDriver                    00013100     example_bufferclass_ctrl_wince.obj
 0002:00000108       splashtex                  00013108     example_bufferclass_draw.obj
 0002:0002abf8       gui32WindowWidth           0003dbf8     wince_unittests.obj
 0002:0002abfc       gui32WindowHeight          0003dbfc     wince_unittests.obj
 0002:0002ac00       gui32PosX                  0003dc00     wince_unittests.obj
 0002:0002ac04       gui32PosY                  0003dc04     wince_unittests.obj
 0002:0002ac08       __security_cookie          0003dc08     corelib0:seccinit.obj
 0002:0002ac0c       __security_cookie_complement 0003dc0c     corelib0:seccinit.obj
 0002:0002ac10       eCameraMode                0003dc10     example_bufferclass_ctrl_wince.obj
 0002:0002ac14       myglTexBindStreamIMG       0003dc14     example_bufferclass_draw.obj
 0002:0002ac18       myglGetTexStreamDeviceAttributeivIMG 0003dc18     example_bufferclass_draw.obj
 0002:0002ac1c       myglGetTexStreamDeviceNameIMG 0003dc1c     example_bufferclass_draw.obj
 0002:0002ac20       dispType                   0003dc20     example_bufferclass_draw.obj
 0002:0002ac24       eglWindow                  0003dc24     example_bufferclass_draw.obj
 0002:0002ac28       gbWindow                   0003dc28     wince_unittests.obj
 0002:0002ac2c       ghWnd                      0003dc2c     wince_unittests.obj
 0002:0002ac30       pfnRegisteredWndProc       0003dc30     wince_unittests.obj
 0002:0002ac34       _exitflag                  0003dc34     corelib0:cexit.obj
 0002:0002ac38       bufferFormat               0003dc38     <common>
 0002:0002ac3c       bufferWidth                0003dc3c     <common>
 0002:0002ac40       context                    0003dc40     <common>
 0002:0002ac44       dpy                        0003dc44     <common>
 0002:0002ac48       bufferHeight               0003dc48     <common>
 0002:0002ac4c       surface                    0003dc4c     <common>
 0002:0002ac50       numBuffers                 0003dc50     <common>
 0002:0002ac54       __onexitend                0003dc54     <common>
 0002:0002ac58       __onexitbegin              0003dc58     <common>

 entry point at        0001:0000152c

 Static symbols

 0001:00000960       init                       00011960 f   example_bufferclass_draw.obj
 0001:00000cf4       handle_egl_error           00011cf4 f   example_bufferclass_draw.obj
 0001:000014b4       WinMainCRTStartupHelper    000124b4 f   corelib0:pegwmain.obj
 0001:00001560       doexit                     00012560 f   corelib0:cexit.obj
